:0300000002000EED
:03000300020028D0
:20000B0002001F758165D2AFD2A912002B80FE12001B80FB758CDC758A00050832050832A0
:20002B007400F511747075F017F55485F055746475F000F54A85F04B795A7A00E98AF0C01C
:20004B00E0C0F0746475F000C0E0C0F0121B3015811581158115811210AC121B66748075F9
:20006B00F025C0E0C0F0121B6915811581798C7A1EE98AF0F9AAF089828A83E493A3F5F0A4
:20008B00E493C5F0C0E0C0F0121B8C158115811207201208891207921206F3120611120423
:2000AB001A1204F91202591202D112031A1209A2120D51120D8A1211B1120F8A12123812C8
:2000CB00127112132C1218851205D802009D227F09121D2D740075F00078FD121D21F60862
:2000EB00A6F0121BB8C0E0C0F0121BA01581158178FC121D21F67B0D7C00121E2D45F07071
:20010B0003020142801678FD121D21E60886F0121DEA18F608A6F0121DF380C678FD121DFC
:20012B0021E60886F079F6121D26121D4378FC121D21E6F702011178FD121D21E60886F01B
:20014B0079F6121D26121D437400F778FD121D21E60886F07B007C00121E2445F0700302D5
:20016B00017574FF75F0FF02018B79F6121D26E98AF0C0E0C0F0121BC81581158102018B73
:20018B007FF7021D3C05810581058105810581740075F00078FD121D21F608A6F078FD122C
:2001AB001D21E60886F07B027C00121E0445F07003020202801678FD121D21E60886F012E6
:2001CB001DEA18F608A6F0121DF380D178FD121D21E60886F079FA121D26121D43C001C00A
:2001EB0002121BB8C0E0C0F0121BA015811581D007D000F60201C178FD121D21E60886F03A
:20020B0079FA121D26121D437400F7740075F00079FA121D26121D43E7C39430121D537BB0
:20022B0004121D4A121DCBC0E0C0F0740175F00079F8121D26121D43E7C39430D004D003C5
:20024B004BC5F04CC5F0121D537FFB021D3CE51575F0007B697C00121E2445F0700302027C
:20026B00D0744A75F020C0E0C0F0121B8C15811581740075F000C0E0C0F01208E11581155C
:20028B0081740475F000C0E0C0F01200DA7B647C00121D5CC0E0C0F0121C2D1581158115E7
:2002AB00811581740475F000C0E0C0F0121C0D15811581F55485F055E5548555F0F55285A6
:2002CB00F05312072022E511540875F0007B007C00121E2D45F07003020319E5528553F0A5
:2002EB00121DF3F55285F053121DEAE5528553F07B007C00121E3E45F07003020319E55446
:20030B008555F0F55285F053E5114404F51122E51614F51604E51675F0007B007C00121EEE
:20032B003E45F070030204197464F516748575F000C0E0C0F0121C3F15811581C0E0C0F033
:20034B00740075F000C0E0C0F0121BFE15811581D004D003121E2445F0602B748375F000FB
:20036B00C0E0C0F0121C3F15811581C0E0C0F0740175F000C0E0C0F0121BFE15811581D0E8
:20038B0004D003121E2445F070030203A8E5114408F511742C75F001F54A85F04B74857517
:2003AB00F000C0E0C0F0121C3F15811581C0E0C0F0740275F000C0E0C0F0121BFE15811508
:2003CB0081D004D003121E2445F0602B748375F000C0E0C0F0121C3F15811581C0E0C0F041
:2003EB00740375F000C0E0C0F0121BFE15811581D004D003121E2445F07003020419E511B7
:20040B0054F7F511746475F000F54A85F04B22E51575F0007B747C00121E2445F07003025A
:20042B0004F8742FF515746375F020C0E0C0F0121B8C15811581748E75F000C0E0C0F0744C
:20044B000075F000C0E0C0F01208921581158115811581748475F000C0E0C0F01201901276
:20046B001D53C0E0C0F01208921581158115811581743A75F000C0E0C0F0121BA0158115D2
:20048B0081748275F000C0E0C0F0120190121D53C0E0C0F012089215811581158115817438
:2004AB003A75F000C0E0C0F0121BA015811581748075F000C0E0C0F0120190121D53C0E0DB
:2004CB00C0F01208921581158115811581748E75F000C0E0C0F0748075F000C0E0C0F012EB
:2004EB000892158115811581158112072022E51575F0007B647C00121E2445F070030205E7
:20050B00D7742FF515747075F020C0E0C0F0121B8C15811581748E75F000C0E0C0F0740083
:20052B0075F000C0E0C0F01208921581158115811581748675F000C0E0C0F0120190121D76
:20054B0053C0E0C0F01208921581158115811581742F75F000C0E0C0F0121BA01581158198
:20056B00748875F000C0E0C0F0120190121D53C0E0C0F01208921581158115811581742FA3
:20058B0075F000C0E0C0F0121BA015811581748C75F000C0E0C0F0120190121D53C0E0C068
:2005AB00F01208921581158115811581748E75F000C0E0C0F0748075F000C0E0C0F01208C2
:2005CB0092158115811581158112072022E51575F0007B0D7C00121E2445F0700302061054
:2005EB00798C7A1EE98AF0F9AAF089828A83E493A3F5F0E493C5F0C0E0C0F0121B8C15817B
:20060B00158112072022E51575F0007B2F7C00121E2445F070030206F2747D75F020C0E04D
:20062B00C0F0748775F000C0E0C0F0121C3F15811581C0E0C0F0748975F000C0E0C0F012A2
:20064B001C3F15811581C0E0C0F0748D75F000C0E0C0F0121C3F15811581C0E0C0F07404A1
:20066B0075F0001218EC7FF8121D2D748E75F020C0E0C0F0748575F000C0E0C0F0121C3F2F
:20068B0015811581C0E0C0F0748375F000C0E0C0F0121C3F15811581C0E0C0F0748175F0E4
:2006AB0000C0E0C0F0121C3F15811581C0E0C0F0740475F0001218EC7FF8121D2D12080A0C
:2006CB00749E75F020C0E0C0F079177A00E98AF0C0E0C0F0740275F0001218EC158115814E
:2006EB001581158112072022E598540175F0007B007C00121E2D45F0700302071B121BB82C
:20070B00C0E0C0F0121BA015811581F51502071F74FFF51522798E7A1EE98AF0F9AAF08996
:20072B00828A83E493A3F5F0E493C5F0C0E0C0F0121B8C158115812205810581740075F0B8
:20074B000078FD121D21F608A6F078FD121D21E60886F078F9121D218603088604121E04FC
:20076B0045F0700302078D801678FD121D21E60886F0121DEA18F608A6F0121DF380CB023D
:20078B00077415811581221207991207D322E5508551F0121DEAF55085F051121DF3E5504F
:2007AB008551F0AB4AAC4B121E4745F070030207D2740075F000F55085F051E5114440F52F
:2007CB0011C2B47405F51422E511544075F0007B007C00121E2D45F07003020809E51414D8
:2007EB00F51404E51475F0007B007C00121E2445F07003020809D2B4E51154BFF5112205C1
:20080B008105810581C2B5C2B4740075F00078FC121D21F608A6F0121CD478FE121D21F664
:20082B007B007C00121E2D45F0700302086B801678FC121D21E60886F0121DEA18F608A6A9
:20084B00F0121DF380D178FC121D21E60886F079177A00121D4378FE121D21E6F702083B9E
:20086B0078FC121D21E60886F079177A00121D437400F7D2B5D2B415811581158122308DB0
:20088B00FDC28D438CDC220581058178F7121D21E6121D5378FD121D21F608A6F018E608A2
:2008AB0086F07B087C00121DCB18F608A6F018E60886F078F9121D214608080808F608A6CB
:2008CB00F018E60886F0C0E0C0F0121C6D15811581158115812278FB121D21E6F513E51393
:2008EB00A2E0929020E106D291C2928004D292C291002205810581740175F000795A7A00FB
:20090B00121D43E775F00078FD121D21F608A6F018E60886F07B087C00121DCB18F608A684
:20092B00F0740075F000795A7A00121D4378FD121D21E60886F04715811581227401255A72
:20094B00F55AE4355BF55BE4355CF55C22120947740275F000795A7A00121D43E775F00049
:20096B00C0E0C0F01208E1158115811208FE2278FB121D21E675F0007B047C00121DD9F6B4
:20098B002430C5F03400C5F02278FB121D21E6540F2430121D5322E511540475F0007B0006
:2009AB007C00121E2D45F07003020D0F12080A120958C0E0C0F0748775F000C0E0C0F012E4
:2009CB001C3F15811581C0E0C0F012097A15811581121D53C0E0C0F0121C1F158115811514
:2009EB00811581120958C0E0C0F0748775F000C0E0C0F0121C3F15811581C0E0C0F012095E
:200A0B009415811581121D53C0E0C0F0121C1F1581158115811581120958C0E0C0F07489D4
:200A2B0075F000C0E0C0F0121C3F15811581C0E0C0F012097A15811581121D53C0E0C0F07A
:200A4B00121C1F1581158115811581120958C0E0C0F0748975F000C0E0C0F0121C3F15816E
:200A6B001581C0E0C0F012099415811581121D53C0E0C0F0121C1F15811581158115811221
:200A8B000958C0E0C0F0748D75F000C0E0C0F0121C3F15811581C0E0C0F012097A158115BB
:200AAB0081121D53C0E0C0F0121C1F1581158115811581120958C0E0C0F0748D75F000C04A
:200ACB00E0C0F0121C3F15811581C0E0C0F012099415811581121D53C0E0C0F0121C1F1583
:200AEB0081158115811581120958C0E0C0F0748575F000C0E0C0F0121C3F15811581C0E0FE
:200B0B00C0F012097A15811581121D53C0E0C0F0121C1F1581158115811581120958C0E0CF
:200B2B00C0F0748575F000C0E0C0F0121C3F15811581C0E0C0F012099415811581121D5306
:200B4B00C0E0C0F0121C1F1581158115811581120958C0E0C0F0748375F000C0E0C0F01214
:200B6B001C3F15811581C0E0C0F012097A15811581121D53C0E0C0F0121C1F158115811572
:200B8B00811581120958C0E0C0F0748375F000C0E0C0F0121C3F15811581C0E0C0F01209C0
:200BAB009415811581121D53C0E0C0F0121C1F1581158115811581120958C0E0C0F074813B
:200BCB0075F000C0E0C0F0121C3F15811581C0E0C0F012097A15811581121D53C0E0C0F0D9
:200BEB00121C1F1581158115811581120958C0E0C0F0748175F000C0E0C0F0121C3F1581D5
:200C0B001581C0E0C0F012099415811581121D53C0E0C0F0121C1F1581158115811581741D
:200C2B000075F000F55885F059E5588559F079177A00121D43E775F0007B007C00121E2D02
:200C4B0045F07003020C8F8012E5588559F0121DEAF55885F059121DF380CE120958C0E0F0
:200C6B00C0F0E5588559F079177A00121D43E775F000C0E0C0F0121C1F1581158115811572
:200C8B0081020C54120958C0E0C0F0740075F000C0E0C0F0121C1F1581158115811581E5F0
:200CAB001154FBF511E54E854FF0121DEAF54E85F04F120D10740075F000C0E0C0F012083A
:200CCB00E115811581740675F000C0E0C0F0E54E854FF0C0E0C0F0121C2D15811581158169
:200CEB00158174A175F020C0E0C0F0E54E854FF0C0E0C0F0740275F0001218EC1581158105
:200D0B001581158122E54E854FF07B887C13121E4745F07003020D50E51154F7F511746454
:200D2B0075F000F54A85F04B743C75F000C0E0C0F074FF75F0FFC0E0C0F0121C1F158115C0
:200D4B00811581158122E51575F0007B727C00121E2445F07003020D8974A475F020C0E020
:200D6B00C0F0E54E854FF0C0E0C0F0740275F0001218EC158115811581158112072022E5E8
:200D8B001575F0007B737C00121E2445F07003020F2D740075F000C0E0C0F01208E1158170
:200DAB00158174BA75F020C0E0C0F0740075F000C0E0C0F0121BFE15811581C0E0C0F0744B
:200DCB000175F000C0E0C0F0121BFE15811581C0E0C0F0740375F0001218EC7FFA121D2DE4
:200DEB00740075F000C0E0C0F0120190121D53C0E0C0F0121C1F1581158115811581743AF7
:200E0B0075F000C0E0C0F0121BA015811581740175F000C0E0C0F0120190121D53C0E0C06A
:200E2B00F0121C1F158115811581158174CD75F020C0E0C0F0740275F000C0E0C0F0121BA4
:200E4B00FE15811581C0E0C0F0740375F000C0E0C0F0121BFE15811581C0E0C0F07403754E
:200E6B00F0001218EC7FFA121D2D740275F000C0E0C0F0120190121D53C0E0C0F0121C1F9F
:200E8B001581158115811581743A75F000C0E0C0F0121BA015811581740375F000C0E0C057
:200EAB00F0120190121D53C0E0C0F0121C1F158115811581158174E075F020C0E0C0F07480
:200ECB000075F000C0E0C0F0121BFE15811581C0E0C0F0740175F000C0E0C0F0121BFE1541
:200EEB00811581C0E0C0F0740275F000C0E0C0F0121BFE15811581C0E0C0F0740375F000D2
:200F0B00C0E0C0F0121BFE15811581C0E0C0F0740575F0001218EC7FF6121D2D120F2E12A9
:200F2B00072022740075F000C0E0C0F0121BFE158115817B997C00121E2445F07003020F40
:200F4B006C743C75F000C0E0C0F0740175F000C0E0C0F0121C1F1581158115811581020FD5
:200F6B0089743C75F000C0E0C0F074FF75F0FFC0E0C0F0121C1F158115811581158122E5A5
:200F8B001575F0007B3D7C00121E2445F070030210AB740075F000C0E0C0F01208E1158125
:200FAB00158174F675F020C0E0C0F0740075F000C0E0C0F0121BFE15811581C0E0C0F0740D
:200FCB000175F000C0E0C0F0121BFE15811581C0E0C0F0740375F0001218EC7FFA121D2DE2
:200FEB00740875F021C0E0C0F0740275F000C0E0C0F0121BFE15811581C0E0C0F0740375D6
:20100B00F000C0E0C0F0121BFE15811581C0E0C0F0740375F0001218EC7FFA121D2D741A89
:20102B0075F021C0E0C0F0740475F000C0E0C0F0121C0D158115817B647C00121D70C0E0A1
:20104B00C0F0740275F0001218EC1581158115811581743C75F000C0E0C0F0121BFE158166
:20106B0015817B017C00121E2445F07003021093743875F021C0E0C0F0740175F0001218B0
:20108B00EC158115810210A8744175F021C0E0C0F0740175F0001218EC1581158112072093
:2010AB0022740075F000C0E0C0F01208E115811581740475F000C0E0C0F0121C0D158115A0
:2010CB0081F55485F055E5548555F0F55285F053740675F000C0E0C0F0121C0D15811581C9
:2010EB00F54E85F04F79607A00E98AF0C0E0C0F0742E75F000C0E0C0F0121B3015811581F8
:20110B0015811581795D7A00E98AF0C0E0C0F0E54E854FF0C0E0C0F0121B301581158115B0
:20112B00811581795D7A00E98AF0C0E0C0F079607A00E98AF0C0E0C0F0121A8215811581AA
:20114B0015811581795D7A00E98AF0C0E0C0F0746475F000C0E0C0F0121B3015811581152A
:20116B0081158179637A00E98AF0C0E0C0F0795D7A00E98AF0C0E0C0F0121A4115811581A8
:20118B0015811581795A7A00E98AF0C0E0C0F079637A00E98AF0C0E0C0F0121AF315811545
:2011AB00811581158122E51575F0007B6E7C00121E2445F07003021237744875F021C0E068
:2011CB00C0F0121B8C15811581121BB87B797C00121E2445F07003021234E51154F7F5118F
:2011EB00740075F000F54E85F04F740675F000C0E0C0F0740075F000C0E0C0F0121C2D153C
:20120B0081158115811581795A7A00E98AF0C0E0C0F0746475F000C0E0C0F0121B30158100
:20122B0015811581158112171B12072022E51575F0007B3F7C00121E2445F070030212702D
:20124B0079907A1EE98AF0F9AAF089828A83E493A3F5F0E493C5F0C0E0C0F0121B8C15810A
:20126B00158112072022E51575F0007B637C00121E2445F0700302132B745B75F021C0E088
:20128B00C0F0748775F000C0E0C0F0121C3F15811581C0E0C0F0748975F000C0E0C0F01236
:2012AB001C3F15811581C0E0C0F0748D75F000C0E0C0F0121C3F15811581C0E0C0F0740435
:2012CB0075F0001218EC7FF8121D2D746D75F021C0E0C0F0748575F000C0E0C0F0121C3FE3
:2012EB0015811581C0E0C0F0748375F000C0E0C0F0121C3F15811581C0E0C0F0748175F078
:20130B0000C0E0C0F0121C3F15811581C0E0C0F0740475F0001218EC7FF8121D2D1207208A
:20132B0022E51575F0007B617C00121E2445F070030214631217EF795D7A00E98AF0C0E0E9
:20134B00C0F0740175F000C0E0C0F0121B301581158115811581795A7A00E98AF0C0E0C0E3
:20136B00F0795D7A00E98AF0C0E0C0F0121A541581158115811581795D7A00E98AF0C0E044
:20138B00C0F0795A7A00E98AF0C0E0C0F0121AF31581158115811581795A7A00E98AF0C0AB
:2013AB00E0C0F0746475F000C0E0C0F0121B301581158115811581795D7A00E98AF0C0E0FD
:2013CB00C0F0795A7A00E98AF0C0E0C0F0121B0E15811581158115817B007C00121E14453F
:2013EB00F07003021460740075F000F55885F059E5588559F07B2E7C00121E3745F07003D6
:20140B000214488012E5588559F0121DEAF55885F059121DF380D9E5588559F079177A0002
:20142B00121D43C001C002120958C0E0C0F0121BFE15811581D007D000F6021410E558850D
:20144B0059F079177A00121D437400F71214641216CF0213C212072022740D75F000C0E018
:20146B00C0F012170915811581740A75F000C0E0C0F012170915811581747D75F021C0E0AB
:20148B00C0F0740075F00079177A00121D43E775F000C0E0C0F0740175F00079177A0012AA
:2014AB001D43E775F000C0E0C0F0740275F00079177A00121D43E775F000C0E0C0F07403BB
:2014CB0075F00079177A00121D43E775F000C0E0C0F0740475F00079177A00121D43E775CF
:2014EB00F000C0E0C0F0740575F00079177A00121D43E775F000C0E0C0F0740775F00012B9
:20150B0018EC7FF2121D2D748C75F021C0E0C0F0740675F00079177A00121D43E775F00072
:20152B00C0E0C0F0740775F00079177A00121D43E775F000C0E0C0F0740875F00079177A6D
:20154B0000121D43E775F000C0E0C0F0740975F00079177A00121D43E775F000C0E0C0F078
:20156B00740A75F00079177A00121D43E775F000C0E0C0F0740B75F00079177A00121D4305
:20158B00E775F000C0E0C0F0740775F0001218EC7FF2121D2D740075F000F55885F059E508
:2015AB00588559F07B187C00121E3745F070030216408014E5588559F02403C5F03400C510
:2015CB00F0F55885F05980D7749C75F021C0E0C0F0E5588559F0240DC5F03400C5F079174E
:2015EB007A00121D43E775F000C0E0C0F0E5588559F0240EC5F03400C5F079177A00121D44
:20160B0043E775F000C0E0C0F0E5588559F0240FC5F03400C5F079177A00121D43E775F03C
:20162B0000C0E0C0F0740475F0001218EC7FF8121D2D0215BF74A475F021C0E0C0F074252C
:20164B0075F00079177A00121D43E775F000C0E0C0F0742675F00079177A00121D43E7752B
:20166B00F000C0E0C0F0742775F00079177A00121D43E775F000C0E0C0F0742875F000798D
:20168B00177A00121D43E775F000C0E0C0F0742975F00079177A00121D43E775F000C0E036
:2016AB00C0F0742A75F00079177A00121D43E775F000C0E0C0F0740775F0001218EC7FF2ED
:2016CB00121D2D220581121CCD7B137C00121E2445F0700302170678FE121D21E6121D53AD
:2016EB007B11121D4A121E2D45F07003021706121CCD78FE121D21F60216E215812278FBDA
:20170B00121D21E6F5133099FDC299E513F5992274B275F021C0E0C0F0121B8C15811581D6
:20172B0079177A00E98AF0C0E0C0F0743275F000C0E0C0F0121CDF158115811581158174AD
:20174B000075F000C0E0C0F01208E115811581740075F000F55885F059E5588559F0791713
:20176B007A00121D43E775F0007B007C00121E2D45F070030217C98012E5588559F0121D7C
:20178B00EAF55885F059121DF380CEE5588559F02408C5F03400C5F0C0E0C0F0E558855989
:2017AB00F079177A00121D43E775F000C0E0C0F0121C1F1581158115811581021784E55897
:2017CB008559F02408C5F03400C5F0C0E0C0F0740075F000C0E0C0F0121C1F15811581155F
:2017EB00811581220581740D75F000C0E0C0F012170915811581740A75F000C0E0C0F01246
:20180B00170915811581740075F000C0E0C0F01208E115811581740075F000F55885F0592D
:20182B00E5588559F02408C5F03400C5F0C0E0C0F0121BFE1581158178FE121D21F67B00EA
:20184B007C00121E2D45F070030218828012E5588559F0121DEAF55885F059121DF380C02D
:20186B0078FE121D21E6121D53C0E0C0F0121BA015811581021859158122740075F000C022
:20188B00E0C0F01208E115811581743C75F000C0E0C0F0121BFE158115817B017C00121EA2
:2018AB002445F070030218EBE5B0540475F0007B007C00121E2445F070030218DBE51144D8
:2018CB0008F511742C75F001F54A85F04B0218EBE51154F7F511746475F000F54A85F04B62
:2018EB002223F42581F8868208868308E4FEFF93700122B42555A3E493B42D06430780A342
:20190B00E493B4300343074024D0B40A00500CCE75F00AA42EFEA3E49380EDE493B4641390
:20192B00E60886F030F708430720121DFAA6F018F68003B4750543070A801CB478054307B6
:20194B00108014B46F0B430708800C121BA6A3809BB462624307027A00C004C005C006C0EE
:20196B0007AB0753031F7C00E60886F0121D98A6F018F6EDD007D006D005D0042430B43A5E
:20198B000040022407C0E00AE645F070CCA902EF30E506742D121BA60A121A22D0E0121B70
:2019AB00A6D9F90808EF30E7A5EAC39E50A07420121BA60A80F3B4630BAA01121A22E612B7
:2019CB001BA680DFB4732BC082C08386820886837A00E4936004A30A80F886831886821237
:2019EB001A22E493A36005121BA680F6D083D08280B1B4691986017A00E76004090A80F9F4
:201A0B00121A228601E7609B121BA60980F7F97A01121A22E980A8EE601B8FF020F716C009
:201A2B0002EAC39E500D742030F6027430121BA60A80EED00222121B4D7A03C3E637F6087D
:201A4B0009DAF9E4F5F092E022121B4D7A03C3E697F60809DAF980EB121B45C37A03E633FB
:201A6B00F608DAFA80DD121B457A03C82AC8C318E613F6DAFA80CC121B4DAB00A8817F03C9
:201A8B00121D2D08AC00121AF6121B59A803121A7450077863A904121A44A803121B0260AF
:201AAB000CA804121A66A804121B0270DFA8037963121AF67FFD021D3C121B4DAB00AC0155
:201ACB00121B597D19C3A803121A67DD0280337863121A677863A904121B1120E7E778634F
:201AEB00A904121A57D380DE121B4D7A03E7F60908DAFA22121B457A0375F000E6700308EA
:201B0B00DAFA22121B4D7A03E82AF8E92AF9181987F0E6B5F006DAF6E4F5F02274FF40F917
:201B2B0004F5F00422E58124FBF98700121B5B87000909E7F60809E7F622E58124FBF88675
:201B4B000022E58124FBF88601181886002278637A03760008DAFB22D2AF22C2AF2278FB06
:201B6B00121D218603088604748075F070121D98121DFA758921F58DF58B75885975985260
:201B8B002278FB121D218682088683E493602D121BA6A380F678FB121D21E63099FDC29982
:201BAB00F599B40A17740D80F2E430980C3098FDC298E599B40D02740A75F0002278FB1222
:201BCB001D218601E4FBFCFFE709B42D030FE709C39430B40A005012FA740A75F000121DD5
:201BEB005C2AFBE5F03400FC80E4EB8CF0DF03021DFA2278FB121D218682088683E075F04B
:201C0B00002278FB121D218682088683E0F5F0A3E0C5F02278F9121D21868208868308E6D4
:201C2B00F02278F9121D21868208868308E608F0A3E6F02278FB121D21C293C295D2931246
:201C4B001CB575F008C3E6139294121C9FD5F0F775F008121CAAA29413D5F0F7C293121C03
:201C6B00B52278FB121D21C293C295D293121CB575F008C308E6139294121C9FD5F0F77576
:201C8B00F008C318E6139294121C9FD5F0F7C293121CB522C295121CB5D295121CB522D2EC
:201CAB0095121CB5C295121CB522C0E07405D5E0FDD0E02278FB121D21E63099FDC299F5E9
:201CCB00992274FFF5F030980A3098FDC298E59975F0002278FB121D21860418188601E408
:201CEB00FD121BB8B408028003B47F16ED60F21D7408121BA67420121BA67408121BA619F3
:201D0B0080DF121BA6F724F36006090DEDB504D1E4F7F5F0ED22C82581C822C92581C97AAC
:201D2B000022D083D082CF2581F581CFC082C08322CF2581F581CF2229F9E5F03AFA227CCB
:201D4B0000CB30E7011CCB2275F00030E70215F022FEEBA4FD8EF0ECA4FCEB8EF0A4C5F091
:201D6B002C2DC5F022C0F0C0E0E5F06C5480FF8CF030F707EB121DFAACF0FBD0E0D0F030CF
:201D8B00F703121DFABF8005121D988062C002C001AAF0F97E007D007F11C3E933F9EA3392
:201DAB00FADF08F5F0E9D001D00222ED33FDEE33FEC3ED9BF5F0EE9C40E0ADF0FED380DBC5
:201DCB00BB000122C333C5F033C5F0DBF722BB000122C3C5F013C5F013DBF722121DEA0451
:201DEB00700205F022121DF314B4FF0215F022121DF3F4C5F0F4C5F022121E574029801E19
:201E0B00121E5740227017801E121E5740107017800C121E5750108005121E6B6009E4F576
:201E2B00F022121E6B60F7E4F5F00422121E6B40F680EB121E6B40EF70E480EB121E6B4004
:201E4B00DD70E480D9121E6B50DD80D2C39BC5F09C20E70720D207C345F02220D2F9D32223
:201E6B00C5F0C39C7003E5F09B22FBE493CB22FCE493FB740193CC22FAE493F9740193CA3F
:201E8B0022921ECD1ED11E0A0A4D696E694C4F474745522056312E3020434F5059524947E8
:201EAB0048542028432920313939392C3230303020574943484954205349524943484F5470
:201ECB0045000A3E3E000A0A48454C50204D454E55202020202020202020202020202020BA
:201EEB00200A2F2072656164206F6E6365202020202020202020202020202020200A74205F
:201F0B0054494D4520736574202020202020202020202020202020200A642044415445204F
:201F2B00736574202020202020202020202020202020200A6320436C6F636B206469737001
:201F4B006C6179202020202020202020202020202020200A732053544152542F53544F5090
:201F6B00207265636F7264696E672074696D65202020202020202020202020202020200AA0
:201F8B006920496E74657276616C202020202020202020202020202020200A3D20736574B5
:201FAB0074696E6720706172616D6574657273202020202020202020202020202020200A06
:201FCB0072206E756D626572206F66207265636F7264202020202020202020202020202087
:201FEB0020200A6720476574207265636F7264202020202020202020202020202020200A3C
:20200B006E204E6577207265636F7264202020202020202020202020202020200A61204192
:20202B004C4C2072656164202020202020202020202020202020200A3F2068656C70000A25
:20204B0020696E74657276616C2031302D36303020736563203E20002048483A4D4D3A53C2
:20206B0053203D20002044442F4D4D2F5952203D20000A253032782F253032782F253032D0
:20208B00782000253032783A253032783A2530327820002569002575000A257520726563E6
:2020AB006F72647320617661696C61626C65000A535441525420253032783A25303278208C
:2020CB003E000A53544F502020253032783A25303278203E000A20253032783A253032782F
:2020EB0020253032783A25303278000A20535441525420253032783A25303278000A2053F0
:20210B00544F502020253032783A25303278000A2053414D504C494E4720494E54455256CC
:20212B00414C2873656329203D202575000A204D414E55414C000A204155544F000A204EA1
:20214B006577207265636F72643F28592F4E29000A20253032782F253032782F253032780E
:20216B002000253032783A253032783A253032782000256325632F256325632F2563256315
:20218B00002C256325633A256325633A25632563002C256325632563002C256325632563DC
:2021AB00256325632563000A3C2D2D20456E746572206465736372697074696F6E20746501
:1B21CB00787420286D61782035302063686172616374657273292D2D3E0A00EF
:00000001FF
